:100000000EC028C027C026C025C024C023C022C0DF
:1000100021C020C01FC01EC01DC01CC01BC0112499
:100020001FBECFE5D2E0DEBFCDBF10E0A0E6B0E05E
:10003000ECE9FFE102C005900D92A238B107D9F7B3
:1000400011E0A2E8B0E001C01D92A931B107E1F7CB
:10005000B5DBA3CFD5CF89E288BB08952091770087
:10006000309178004091790050917A000DDF20E0C6
:1000700030E040E050E004C02F5F3F4F4F4F5F4FF4
:100080006217730784079507BCF72093D500309358
:10009000D6004093D7005093D800089589E288BBDA
:1000A00061E070E080E090E0D9DF88E288BB0895ED
:1000B00020917B0030917C0040917D0050917E002A
:1000C000E3DE20E030E040E050E004C02F5F3F4F2F
:1000D0004F4F5F4F6217730784079507BCF7209354
:1000E000D9003093DA004093DB005093DC00089590
:1000F0001F9318BA81E087BB19E218BB68EE73E062
:1001000080E090E0ABDF83E087BB18BB61E070E08C
:1001100080E090E0A3DF1F91089583E087BB89E230
:1001200088BB0895662391F4853011F417B83EC05A
:10013000823011F481E039C0843011F482E035C09E
:10014000833099F18A3091F58DE02FC06130A1F4B0
:10015000853011F480E929C0823011F481E925C08D
:10016000843011F482E921C0833011F483E91DC089
:100170008A30E1F48DE919C06230C1F4853011F4A0
:1001800080E813C0823011F481E80FC0843011F48C
:1001900082E80BC0833011F483E807C08A3011F481
:1001A0008DE803C08B3011F48FE887B986EC86B9EF
:1001B0003699FECF84B195B19C0140E050E0209388
:1001C000AD003093AE004093AF005093B000662373
:1001D00019F58091B5009091B600A091B700B0914B
:1001E000B800281B390B4A0B5B0B2093AD003093F2
:1001F000AE004093AF005093B00057FF08C010927C
:10020000AD001092AE001092AF001092B00020E24C
:100210003EE440E050E05AC06130A1F58091B90061
:100220009091BA00A091BB00B091BC00281B390B83
:100230004A0B5B0B2093AD003093AE004093AF00B0
:100240005093B00057FF08C01092AD001092AE005E
:100250001092AF001092B0002AE030E040E050E091
:100260006091AD007091AE008091AF009091B000B0
:100270000BDE6093AD007093AE008093AF0090935F
:10028000B0003AC06230C1F58091BD009091BE00CF
:10029000A091BF00B091C000281B390B4A0B5B0B2B
:1002A0002093AD003093AE004093AF005093B00068
:1002B00057FF08C01092AD001092AE001092AF0030
:1002C0001092B0002CE434E040E050E06091AD00CA
:1002D0007091AE008091AF009091B000D5DD2FEF0E
:1002E00033E040E050E008DE2093AD003093AE00F4
:1002F0004093AF005093B0006091AD007091AE009C
:100300008091AF009091B00008951092B5001092C6
:10031000B6001092B7001092B80060E08AE002DFE9
:1003200084B195B1A0E0B0E08093B5009093B600A1
:10033000A093B700B093B8001092B9001092BA0021
:100340001092BB001092BC0061E08AE0EBDE84B149
:1003500095B1A0E0B0E08093B9009093BA00A0936B
:10036000BB00B093BC001092BD001092BE00109272
:10037000BF001092C00062E08AE0D4DE84B195B183
:10038000A0E0B0E08093BD009093BE00A093BF00BA
:10039000B093C000089589E288BB61E070E080E01E
:1003A00090E05CDE1092A0001092A1001092A200DA
:1003B0001092A30021C08BE288BB64E170E080E072
:1003C00090E076DE89E288BB69E170E080E090E051
:1003D00045DE8091A0009091A100A091A200B09173
:1003E000A3000196A11DB11D8093A0009093A100D0
:1003F000A093A200B093A3008091A0009091A100CF
:10040000A091A200B091A3000A97A105B1059CF2AA
:1004100008951F93182F109218010BC0BCDF6AEFCC
:1004200070E080E090E01ADE809118018F5F809389
:10043000180180911801811788F31F910895E1999F
:10044000FECF1CBA90E09FBB8EBB6DBBE29AE19AD7
:100450000895E199FECF90E09FBB8EBBE09A8DB3EB
:1004600090E008956F927F928F929F92AF92BF9289
:10047000CF92DF92EF92FF920F931F9361E380E0A0
:10048000DEDF81E0E6DF8F3F21F081E0E2DF809375
:10049000800082E0DEDF8F3F69F082E0DADF90E00B
:1004A000A0E0B0E080936A0090936B00A0936C0092
:1004B000B0936D0083E0CDDF8F3F09F46BC083E024
:1004C000C8DF682E77248824992460926F00709288
:1004D000700080927100909272001092DD00109274
:1004E000DE001092DF001092E000E0906A00F090D1
:1004F0006B0000916C0010916D00EE0CFF1C001F52
:10050000111F84E690E0A0E0B0E0E80EF91E0A1F9B
:100510001B1FE0928B00F0928C0000938D001093D3
:100520008E0025E730E040E050E0C801B701ACDCC8
:10053000A4019301A9DC20EE3EE240E050E0DCDCC7
:1005400059016A0125E230E040E050E0C801B701FE
:100550009BDC64577E408040904028E730E040E0DC
:1005600050E0CADCA20EB31EC41ED51EA0927300BA
:10057000B0927400C0927500D09276008091800095
:10058000833041F460927300709274008092750021
:100590009092760084E05DDF80936E0085E059DF05
:1005A0008F3F91F085E055DF90E064E670E05ADC23
:1005B000AA2797FDA095BA2F809387009093880073
:1005C000A0938900B0938A0080E143DF8F3F21F040
:1005D00080E13FDF80930B0181E13BDF8F3F21F022
:1005E00081E137DF8093100180E233DF8F3F21F01C
:1005F00080E22FDF8093820081E22BDF8F3F21F0AA
:1006000081E227DF8093600082E223DF8F3F21F0C9
:1006100082E21FDF8093610083E21BDF8F3F91F056
:1006200083E217DF90E064E670E01CDCAA2797FD08
:10063000A095BA2F8093830090938400A0938500A7
:10064000B09386001F910F91FF90EF90DF90CF90B5
:10065000BF90AF909F908F907F906F9008956F9212
:100660007F928F929F92AF92BF92CF92DF92EF9242
:10067000FF920F931F933B014C018091DD009091FD
:10068000DE00A091DF00B091E0000196A11DB11D38
:100690008093DD009093DE00A093DF00B093E00034
:1006A00083309105A105B10549F460926F00709205
:1006B0007000809271009092720036C00497A1057C
:1006C000B10594F1E0906F00F0907000009171001E
:1006D000109172002BE030E040E050E0C801B7011B
:1006E000D3DB2AE030E040E050E006DC2615370599
:1006F000480559050CF41BC1C801B701F3E0660FAA
:10070000771F881F991FFA95D1F76E0D7F1D801FE7
:10071000911F2AE030E040E050E0EEDB6216730605
:10072000840695063CF503C120916F00309170005E
:100730004091710050917200CA01B901E2E0660F68
:10074000771F881F991FEA95D1F7620F731F841FC7
:10075000951F660D771D881D991D26E030E040E04D
:1007600050E0CADB20936F0030937000409371001B
:1007700050937200E0906A00F0906B0000916C0062
:1007800010916D00EE0CFF1C001F111F84E690E01D
:10079000A0E0B0E0E80EF91E0A1F1B1FE0928B00DC
:1007A000F0928C0000938D0010938E0060906F008B
:1007B00070907000809071009090720025E230E09F
:1007C00040E050E0C801B7015FDB64577E408040E5
:1007D000904028E730E040E050E08EDB59016A01AC
:1007E00025E730E040E050E0C401B3014DDBA80153
:1007F00097014ADB20EE3EE240E050E07DDB2A0D2F
:100800003B1D4C1D5D1D209373003093740040937D
:10081000750050937600261537054805590544F4B0
:1008200060927300709274008092750090927600CE
:1008300097FE0CC081E090E0A0E0B0E080936F00F4
:1008400090937000A0937100B093720080916F003C
:1008500090917000A0917100B09172008F3F91054E
:10086000A105B10564F08EEF90E0A0E0B0E08093C8
:100870006F0090937000A0937100B093720020916C
:100880006F00309170004091710050917200809122
:100890008F0090919000A0919100B0919200281744
:1008A00039074A075B0799F0622F83E0C8DD809122
:1008B0006F0090917000A0917100B09172008093D0
:1008C0008F0090939000A0939100B093920080913C
:1008D000DD009091DE00A091DF00B091E000039771
:1008E000A105B1056CF480916F0090917000A0910A
:1008F0007100B0917200880F991FAA1FBB1F0FC013
:1009000080918000833099F480916F009091700005
:10091000A0917100B09172000297A109B109809372
:10092000730090937400A0937500B09376001F91AC
:100930000F91FF90EF90DF90CF90BF90AF909F907E
:100940008F907F906F900895982F882339F483E0DB
:100950008ABD80E88CBD89E288BB089581E88CBDA2
:1009600083E28ABD81E083BF92BF98BD88E089BFE2
:100970001CBC089580E0E8DF08951F93182F105CD9
:10098000812F67DD8F5F8093FB008B3F18F08AEF2C
:100990008093FB006091FB00812F51DD1F91089532
:1009A0001F9360E084E0BEDB6093F4007093F50079
:1009B0008093F6009093F700685271418040904018
:1009C000615D73408040904008F0E0C080E0D5DF7A
:1009D0008BE287BB81E088BB11E01093F80018BB65
:1009E00060ED77E080E090E039DB60E084E09ADB66
:1009F0006093F4007093F5008093F6009093F700F5
:100A00006E577241804090406452714080409040E7
:100A100018F082E08093F80061E084E083DB60936B
:100A2000F4007093F5008093F6009093F7006E57F2
:100A3000724180409040645271408040904018F074
:100A400083E08093F80061E082E06CDB6093F40067
:100A50007093F5008093F6009093F7006E57724103
:100A600080409040645271408040904018F084E093
:100A70008093F80083E088BB61E070E080E090E064
:100A8000EDDA61E082E04EDB6093F4007093F500F4
:100A90008093F6009093F7006B3071058105910506
:100AA00018F085E08093F80018BB61E070E080E00A
:100AB00090E0D4DA18BA61E070E080E090E0CEDA3D
:100AC00061E082E02FDB6093F4007093F500809387
:100AD000F6009093F700655E75428040904069553E
:100AE00072408040904018F086E08093F80018BB78
:100AF00061E070E080E090E0B1DA1092F90013C09C
:100B000081E288BB64EF71E080E090E0A7DA81E0E9
:100B100088BB64EF71E080E090E0A0DA8091F9009A
:100B20008F5F8093F9009091F8008091F900891708
:100B300038F39130B9F06CED75E080E090E08EDA3A
:100B400081E288BB6091F4007091F5008091F6001D
:100B50009091F70083DA81E088BB60ED77E080E078
:100B600090E07CDA6091820080E269DC6091600054
:100B700081E265DC6091610082E261DC809183004A
:100B800064E69BD9682F83E25ADC26CF1F91089533
:100B90002F923F924F925F926F927F928F929F928D
:100BA000AF92BF92CF92DF92EF92FF920F931F937B
:100BB00019E218BB61E070E080E090E04FDA8BE270
:100BC00088BB61E070E080E090E048DA61E082E0BC
:100BD000A9DA28EE33E040E050E056D922E03BE0CD
:100BE00040E050E089D920939800309399004093D9
:100BF0009A0050939B0018BB2B3F310541055105CE
:100C00003CF018BB82E0B9DE81E18093930073C0B1
:100C100081E09ADE8091610010916E00813009F0D0
:100C200049C0812F8695282E3324442455242091B1
:100C3000F0003091F1004091F2005091F300612EEC
:100C4000772488249924EE24FF248701AA24BB2436
:100C5000650115C0C601B5016619770988099909AA
:100C600024E630E040E050E047D9220D331D441D1A
:100C7000551D28BD0894E11CF11C011D111DA60C79
:100C8000B71CC81CD91C83E3E816F1040105110543
:100C90000CF32093F0003093F1004093F200509356
:100CA000F300E092EC00F092ED000093EE00109360
:100CB000EF0021C0612F70E080E090E02091EC0017
:100CC0003091ED004091EE005091EF00DDD824E628
:100CD00030E040E050E010D9812F8695280F311D7B
:100CE000411D511D2093F0003093F1004093F2001C
:100CF0005093F30018BD1F910F91FF90EF90DF907C
:100D0000CF90BF90AF909F908F907F906F905F90AB
:100D10004F903F902F90089589E288BB61E070E08A
:100D200080E090E09BD960E083E0FCD924E030E0F3
:100D300040E050E0E1D82093FD003093FE00409366
:100D4000FF005093000160E085E0ECD924E030E042
:100D500040E050E0D1D8209301013093020140934C
:100D60000301509304018091FD009091FE00A09139
:100D7000FF00B09100018C3261E0960760E0A607A9
:100D800060E0B60774F42C3261E0360760E0460795
:100D900060E0560734F481E08093050181E090E043
:100DA0000895255F3140404050401CF083E090E0C2
:100DB0000895855F9140A040B0401CF082E090E033
:100DC000089581E090E00895E6DA80E242DB823027
:100DD00019F060E080E233DB109216011092B1004E
:100DE0001092B2001092B3001092B4004DC060E0B7
:100DF00084E098D9645F71408040904014F4109270
:100E0000C90060E084E08ED92091660030916700CF
:100E10004091680050916900261737074807590725
:100E200004F58091C9008823E1F480E212DB882375
:100E300019F461E080E203DB809116018F5F8093FB
:100E400016018A3019F462E080E2F9DA1092B100FA
:100E50001092B2001092B3001092B40081E080931F
:100E6000C9008091B1009091B200A091B300B091FF
:100E7000B4000196A11DB11D8093B1009093B20002
:100E8000A093B300B093B4008091B1009091B200F0
:100E9000A091B300B091B40088559240A040B040FA
:100EA0000CF4A5CF81E0B5DA76DA61E081E2C7DA49
:100EB0001092B1001092B2001092B3001092B400E0
:100EC0003FC060E084E02ED9645F71408040904074
:100ED00014F41092C90060E084E024D920916600E7
:100EE00030916700409168005091690026173707DC
:100EF0004807590794F48091C900882371F460E091
:100F000081E29DDA1092B1001092B2001092B3000B
:100F10001092B40081E08093C9008091B10090915B
:100F2000B200A091B300B091B4000196A11DB11D13
:100F30008093B1009093B200A093B300B093B4003B
:100F40008091B1009091B200A091B300B091B40033
:100F500088559240A040B0400CF4B3CF82E059DAFB
:100F60001ADA61E082E26BDA1092B1001092B200FC
:100F70001092B3001092B4003FC060E084E0D2D879
:100F8000645F71408040904014F41092C90060E0AA
:100F900084E0C8D8209166003091670040916800D5
:100FA00050916900261737074807590794F4809134
:100FB000C900882371F460E082E241DA1092B10046
:100FC0001092B2001092B3001092B40081E08093AE
:100FD000C9008091B1009091B200A091B300B0918E
:100FE000B4000196A11DB11D8093B1009093B20091
:100FF000A093B300B093B4008091B1009091B2007F
:10100000A091B300B091B40088559240A040B04088
:101010000CF4B3CF83E0FDD9BED960E083E20FDAF0
:10102000109216011092B1001092B2001092B3000B
:101030001092B4004BC060E084E074D8645F7140EB
:101040008040904014F41092C90060E084E06AD8B7
:1010500020916600309167004091680050916900CE
:101060002617370748075907F4F48091C9008823E9
:10107000D1F48091160190E065E070E0F3D68A5BD0
:10108000682F83E2DCD9809116018F5F809316016F
:101090001092B1001092B2001092B3001092B400FE
:1010A00081E08093C9008091B1009091B200A0913D
:1010B000B300B091B4000196A11DB11D8093B100A1
:1010C0009093B200A093B300B093B4008091B100AC
:1010D0009091B200A091B300B091B40088559240B5
:1010E000A040B0400CF4A7CF089564EF71E080E019
:1010F00090E0B4D750D91092E6001092E700109219
:10110000E8001092E9001092B1001092B200109223
:10111000B3001092B40056C060E084E003D8645F6E
:1011200071408040904014F41092C90060E084E067
:10113000F9D7209166003091670040916800509186
:10114000690026173707480759074CF58091C900F1
:10115000882329F58091E6009091E700A091E800AE
:10116000B091E9000196A11DB11D8093E600909316
:10117000E700A093E800B093E900809380008430FA
:1011800018F083E0809380001092B1001092B200BA
:101190001092B3001092B40081E08093C900809156
:1011A000B1009091B200A091B300B091B40001964B
:1011B000A11DB11D8093B1009093B200A093B30024
:1011C000B093B4008091B1009091B200A091B300AF
:1011D000B091B40088559240A040B0400CF49CCF30
:1011E00081E017D9D8D81092B1001092B2001092B5
:1011F000B3001092B40054C060E084E093D7645F01
:1012000071408040904014F41092C90060E084E086
:1012100089D7209166003091670040916800509115
:10122000690026173707480759073CF58091C90020
:10123000882319F580916A0090916B00A0916C0051
:10124000B0916D00181619061A061B06B4F4019722
:10125000A109B10980936A0090936B00A0936C0080
:10126000B0936D001092B1001092B2001092B300D2
:101270001092B40081E08093C9008091B1009091F8
:10128000B200A091B300B091B4000196A11DB11DB0
:101290008093B1009093B200A093B300B093B400D8
:1012A0008091B1009091B200A091B300B091B400D0
:1012B00088559240A040B0400CF49ECF82E0A9D85F
:1012C0006AD81092B1001092B2001092B30010923E
:1012D000B40054C060E084E025D7645F7140804072
:1012E000904014F41092C90060E084E01BD7209174
:1012F00066003091670040916800509169002617A0
:101300003707480759073CF58091C900882319F52C
:1013100080916A0090916B00A0916C00B0916D007B
:101320008A3F9105A105B105B4F40196A11DB11D37
:1013300080936A0090936B00A0936C00B0936D0053
:101340001092B1001092B2001092B3001092B4004B
:1013500081E08093C9008091B1009091B200A0918A
:10136000B300B091B4000196A11DB11D8093B100EE
:101370009093B200A093B300B093B4008091B100F9
:101380009091B200A091B300B091B4008855924002
:10139000A040B0400CF49ECF83E03BD8FCD7109225
:1013A000B1001092B2001092B3001092B40051C07C
:1013B00060E084E0B7D6645F71408040904014F4F0
:1013C0001092C90060E084E0ADD6209166003091B3
:1013D0006700409168005091690026173707480759
:1013E000590724F58091C900882301F580916E008A
:1013F0008823E1F090E069E070E034D56AE070E0C5
:1014000068D560936E001092B1001092B2001092F5
:10141000B3001092B4001092DD001092DE00109222
:10142000DF001092E00081E08093C9008091B1005C
:101430009091B200A091B300B091B4000196A11DAB
:10144000B11D8093B1009093B200A093B300B0930C
:10145000B4008091B1009091B200A091B300B0911E
:10146000B40088559240A040B0400CF4A1CF84E075
:10147000D0D791D71092B1001092B2001092B30061
:101480001092B40057C060E084E04CD6645F7140B5
:101490008040904014F41092C90060E084E042D68D
:1014A000209166003091670040916800509169007A
:1014B000261737074807590754F58091C900882334
:1014C00031F580916E008F3F11F1883E50F490E02D
:1014D0006BE070E0C7D46AE070E0FBD460936E000C
:1014E00003C08EEF80936E001092B1001092B20094
:1014F0001092B3001092B4001092DD001092DE0042
:101500001092DF001092E00081E08093C90080918A
:10151000B1009091B200A091B300B091B4000196D7
:10152000A11DB11D8093B1009093B200A093B300B0
:10153000B093B4008091B1009091B200A091B3003B
:10154000B091B40088559240A040B0400CF49BCFBD
:101550006091800081E073D780916A0090916B0068
:10156000A0916C00B0916D00C297A105B10564F423
:1015700082E390E0A0E0B0E080936A0090936B007B
:10158000A0936C00B0936D0080916A0090916B0005
:10159000A0916C00B0916D008B3F9105A105B10544
:1015A00064F08AEF90E0A0E0B0E080936A0090934E
:1015B0006B00A0936C00B0936D0060916A0082E0B4
:1015C0003ED780916E00843318F484E380936E00DC
:1015D00080916E008F3F19F48EEF80936E006091C2
:1015E0006E0084E02CD76091870070918800809114
:1015F000890090918A0024E630E040E050E07CD4FD
:101600002093EA00622F85E01AD785E002D7C3D67F
:101610001092E2001092E3001092E4001092E500B4
:101620001092B1001092B2001092B3001092B40068
:10163000B7C08091E2009091E300A091E400B091E6
:10164000E5000196A11DB11D8093E2009093E30097
:10165000A093E400B093E5008D5D9540A040B040BC
:101660000CF47AC06FEF80E0EAD66FEF81E0E7D646
:101670006FEF82E0E4D66FEF83E0E1D66FEF84E0B6
:10168000DED66FEF85E0DBD686D685D684D683D6C8
:1016900082D681D680D67FD67ED67DD61092160190
:1016A0001092B1001092B2001092B3001092B400E8
:1016B00044C060E084E036D5645F71408040904073
:1016C00014F41092C90060E084E02CD520916600EB
:1016D00030916700409168005091690026173707E4
:1016E00048075907BCF48091C900882399F4809178
:1016F00016018F5F809316018A3009F465DB109222
:10170000B1001092B2001092B3001092B40081E0C8
:101710008093C9008091B1009091B200A091B30074
:10172000B091B4000196A11DB11D8093B1009093BA
:10173000B200A093B300B093B4008091B100909137
:10174000B200A091B300B091B40088559240A0407F
:10175000B0400CF4AECFFFCF60E084E0E3D4209142
:10176000660030916700409168005091690026172B
:101770003707480759070CF45CCF8091B10090916E
:10178000B200A091B300B091B4000196A11DB11DAB
:101790008093B1009093B200A093B300B093B400D3
:1017A0008091B1009091B200A091B300B091B400CB
:1017B00088559240A040B0407CF20895EF92FF928D
:1017C0000F931F9360ED77E080E090E047D481E0D5
:1017D0008093930080937F0098D560E084E0A2D44A
:1017E000655F7140804090401CF084E080939300DE
:1017F00039D67ED413E017BB89E288BB60E082E073
:1018000091D49B01AC0160939C0070939D008093E8
:101810009E0090939F0028358BE1380780E04807B1
:1018200080E058071CF482E08093930021583E43E7
:101830004040504024F081E0A0D810939300809164
:10184000870090918800A0918900B0918A0000974C
:10185000A105B10559F460E082E064D4609387008B
:10186000709388008093890090938A008091830010
:1018700090918400A0918500B09186000097A10509
:10188000B10541F08093870090938800A093890070
:10189000B0938A00E0908700F09088000091890062
:1018A00010918A0020E530E040E050E0C801B70127
:1018B000EBD224E630E040E050E01ED320936600F7
:1018C00030936700409368005093690025E530E04D
:1018D00040E050E0C801B701D7D224E630E040E054
:1018E00050E00AD320936200309363004093640079
:1018F0005093650011DA8093FC001092D100109291
:10190000D2001092D3001092D40019C064EF71E09D
:1019100080E090E0A3D33FD58091D1009091D20098
:10192000A091D300B091D4000196A11DB11D809368
:10193000D1009093D200A093D300B093D4008091B3
:10194000930090E0A0E0B0E02091D1003091D2006F
:101950004091D3005091D400281739074A075B07FC
:10196000ACF21ED8809193008230F0F71092B10053
:101970001092B2001092B3001092B4001CC060E04C
:1019800084E0D0D369557B41804090400CF0ADDBC2
:101990008091B1009091B200A091B300B091B400D9
:1019A0000196A11DB11D8093B1009093B200A09348
:1019B000B300B093B4008091B1009091B200A091B7
:1019C000B300B091B400815A9440A040B040BCF242
:1019D00080918200882319F083E080938000DBD41B
:1019E000DAD4D9D4D8D480910501882321F0D3D476
:1019F000D2D4D1D4D0D48091CA009091CB00A09100
:101A0000CC00B091CD000196A11DB11D8093CA00FC
:101A10009093CB00A093CC00B093CD0080910701B0
:101A200090910801A0910901B0910A010196A11DB0
:101A3000B11D8093070190930801A0930901B09311
:101A40000A0198D760E084E06DD39B01AC016093FC
:101A500094007093950080939600909397008091E6
:101A6000660090916700A0916800B09169008217AC
:101A70009307A407B507ECF58091C9008823C9F541
:101A8000809105018823A9F4809162009091630000
:101A9000A0916400B0916500281739074A075B07D9
:101AA0006CF48091EB008F5F8093EB008330E8F45F
:101AB000B6C032D98093FC00813019F41092EB004B
:101AC000AEC09091EB009F5F9093EB00833039F4B0
:101AD000933008F4A4C080E1809393001AC182304F
:101AE00009F09DC0933008F49AC080E18093930080
:101AF00096C0245F3140404050406CF41092C900C1
:101B000081E080937F001092CA001092CB00109267
:101B1000CC001092CD008091CA009091CB00A09192
:101B2000CC00B091CD00833A9105A105B10584F0B8
:101B30008091C900813061F480918000833041F050
:101B400080916000813021F482E080937F0067C043
:101B500080910601882309F04ECF8091C1009091B9
:101B6000C200A091C300B091C4008D529140A0402A
:101B7000B04008F440CF8091070190910801A091F6
:101B80000901B0910A01895E9340A040B0400CF475
:101B900032CF8091830090918400A0918500B09114
:101BA00086000097A105B10509F425CF60E082E029
:101BB000B9D27B018C016093870070938800809379
:101BC000890090938A0020E530E040E050E05CD14D
:101BD00024E630E040E050E08FD12093660030935F
:101BE0006700409368005093690025E530E040E0CD
:101BF00050E0C801B70148D124E630E040E050E0B1
:101C00007BD1209362003093630040936400509333
:101C1000650084E0B2D681E080930601ECCE80912D
:101C20001101813009F475C0B3D761E070E080E044
:101C300090E014D21092C5001092C6001092C70016
:101C40001092C8008091C1009091C200A091C30081
:101C5000B091C4000196A11DB11D8093C100909365
:101C6000C200A093C300B093C4008091C5009091BE
:101C7000C600A091C700B091C8000196A11DB11D7A
:101C80008093C5009093C600A093C700B093C8008E
:101C900061E084E047D26093940070939500809354
:101CA000960090939700685B7B408040904084F45E
:101CB00080918000813021F080917F00823021F47A
:101CC00081E080937F0025C08091C900882309F1BD
:101CD00080917F00823049F280918000813029F22A
:101CE0002091C5003091C6004091C7005091C800B6
:101CF0008091730090917400A0917500B09176006E
:101D000082179307A407B5070CF0AFCF81E080934B
:101D1000C90030D6C3D16BE470E080E090E09ED182
:101D200089E288BB8091C900882349F46091C5008D
:101D30007091C6008091C7009091C80090D462E075
:101D40008BE0F0D124E630E040E050E09DD06856D2
:101D50007447804090402DE630E040E050E0CCD029
:101D600020930C0130930D0140930E0150930F010D
:101D70002C333105410551052CF083E0FED581E07F
:101D80008093110120910C0130910D0140910E01C1
:101D900050910F01283331054105510514F410927B
:101DA000110180911101813019F482E18093930037
:101DB0001092CA001092CB001092CC001092CD006D
:101DC00010920701109208011092090110920A0165
:101DD00080910B0190E0A0E0B0E082179307A40788
:101DE000B5072CF420930B01622F80E128D360917A
:101DF00098007091990080919A0090919B002AE040
:101E000030E040E050E078D08091100190E0A0E018
:101E1000B0E082179307A407B5072CF420931001B4
:101E2000622F81E10CD380919300882309F4E3CDE4
:101E300064E670E080E090E011D180919300803101
:101E400011F481E0E6D280919300813111F482E0B7
:101E5000E0D280919300823111F483E0DAD21092C3
:101E60009300C9CD5527002480FF02C0060E571FDE
:101E7000660F771F6115710521F09695879500977C
:101E800099F7952F802D0895FF27EE27BB27AA27C6
:101E900060FF04C0A20FB31FE41FF51F220F331F02
:101EA000441F551F969587957795679589F70097F5
:101EB000760771F7CF01BD010895991B79E004C041
:101EC000991F961708F0961B881F7A95C9F7809579
:101ED000089597FB092E07260AD077FD04D027D056
:101EE00006D000201AF4709561957F4F0895F6F79B
:101EF000909581959F4F089597FB092E05260ED04A
:101F000057FD04D028D00AD0001C38F450954095D5
:101F1000309521953F4F4F4F5F4F0895F6F79095BD
:101F20008095709561957F4F8F4F9F4F0895AA1BA5
:101F3000BB1B51E107C0AA1FBB1FA617B70710F0B4
:101F4000A61BB70B881F991F5A95A9F780959095E6
:101F5000BC01CD010895A1E21A2EAA1BBB1BFD01F5
:101F60000DC0AA1FBB1FEE1FFF1FA217B307E40778
:101F7000F50720F0A21BB30BE40BF50B661F771FD0
:101F8000881F991F1A9469F76095709580959095B0
:0C1F90009B01AC01BD01CF010895FFCF03
:101F9C0001017C1500007017000050000000FE4687
:101FAC00000000CD000000640000000100000001F2
:021FBC00020021
:00000001FF
